:10000000ABC0C5C08ECCC3C0C2C0C1C0C0C0BFC021
:100010003BCCBDC0BCC0BBC075CCB9C0B8C03230D1
:1000200032313035313430363131000000000000DB
:1000300000000000000000000000000000000000C0
:1000400000000000000000000000000000000000B0
:1000500000000000000000000000000000000000A0
:100060000000000000000000000000000001030488
:10007000050708090B0C0E0F1113141618191B1D78
:100080001F21232527292B2D30323437393B3E4081
:100090004346484B4E5154575A5D606366696D70D4
:1000A00073777A7E8185898D9094989CA0A5A9AD5F
:1000B000B1B6BABFC3C8CDD1D6DBE0E5EAEFF4FAFA
:1000C000FF010102020303040405060708090A0CE4
:1000D0000D0E0F11131416181A1D1F2224272A2D76
:1000E0003033373B3E42464B4F54595D63686E7325
:1000F000797F868C939AA1A8B0B8C0C8D1D9E2EC18
:10010000F5FFFFFFFFFFFFFFFFFFFFFFFFFFFFFF09
:10011000FFFFFFFFFFFFFFFFFFFFFFFFFFFFFFFFEF
:10012000FFFFFFFFFFFFFFFFFFFFFFFFFFFFFFFFDF
:10013000FFFFFFFFFFFFFFFFFFFFFFFFFFFFFFFFCF
:10014000FFFFFFFFFFFFFFFFFFFFFFFFFFFFFFFFBF
:10015000FFFFFFFFFFFF000011241FBECFE5D2E02D
:10016000DEBFCDBF10E0A0E6B0E0EAE8FEE102C0ED
:1001700005900D92A439B107D9F721E0A4E9B0E0C8
:1001800001C01D92A833B207E1F7DADB7CCE38CF8D
:10019000482F9B01E5E0F1E080E090E0508155239D
:1001A00031F00196339680319105C1F709C063E0C3
:1001B00070E00BDEFC01EB5FFE4F40833283218356
:1001C00008950F931F93CF93DF93D0910501DD2303
:1001D00051F10091060110910701C091E200C15058
:1001E000C7FD0DC0EC2FEE0FFF0BED51FF4F01903F
:1001F000F081E02DB8018D2F09958111F0CFE5E058
:10020000F1E0838180838481958192838183339619
:1002100081E0E233F807A9F710923201109234011D
:1002200010923301D2CFDF91CF911F910F9108959A
:10023000BC0180913701ACCF10923701109236018A
:100240001092350181E08093C000089590E822E08B
:1002500048EA57E030E0815070F00FB6F89496BD50
:1002600026BD0FBEFA013197F1F70FB6F89496BD8F
:1002700036BD0FBEF0CF089586B383FB882780F983
:1002800091E089278093DB000895E0916600F0916A
:1002900067003196FB70F460F0936700E0936600AE
:1002A0008091D7008B5A8093D700E4918091D7003A
:1002B0008E0F0895CF93DF9300D000D000D0CDB73C
:1002C000DEB79091BC002091F3003091F400235AE6
:1002D000374009F492E06623F9F0823019F427E9F7
:1002E000261B622F26E0EEE7F0E0DE01119601907A
:1002F0000D922A95E1F7E82FF0E03197EE0FFF1FFE
:1003000021E030E02C0F3D1FE20FF31F0190F08140
:10031000E02DE90FF11D608326960FB6F894DEBF3D
:100320000FBECDBFDF91CF910895813019F41092A7
:10033000BE0008956093BD000895BF92CF92DF92F2
:10034000EF92FF920F931F93CF93DF93EC014091B5
:10035000BC00E0917900EE2311F082E001C0842F0F
:1003600090E0DC01AC58BF4F2C9120937800DC0169
:10037000AF58BF4F8C9180937700F0E0E259FF4F68
:100380003181622F70E0442349F0313039F49B0110
:10039000280F311DC9019595879536C0C617D70717
:1003A00094F1682F70E06C177D0774F1411102C061
:1003B0008C2F2AC0821B032F10E001501109E82E58
:1003C000F12CC701B80132DD6093BB006695E62FC2
:1003D000F0E0822FC12CD12CB12CB316A9F0C601AC
:1003E000B80110DD822F860FCE0CDF1CAE01481B3A
:1003F000510957FF03C0519541955109E417F5077D
:100400001CF4B394EACF822FDF91CF911F910F910B
:10041000FF90EF90DF90CF90BF90089581E0089516
:10042000611160937C000895662389F0813061F446
:100430008091F6009091F500891B681B6093F50090
:1004400082E080937D0003C0635E60937B008091B7
:100450007B00873418F086E480937B0008956093D6
:10046000B60008950F931F93CF93DF938091BC0044
:100470008093C100809174008093C20080917100CC
:100480008093C300809175008093C40080917200B6
:100490008093C50080916F008093C6008091BE005C
:1004A0008093C7008091BD008093C80080916B004D
:1004B0008093C900809169008093CA0080916A008E
:1004C0008093CB00809168008093CC0080916C0079
:1004D0008093CD00809179008093CE00809176004A
:1004E0008093CF00809173008093D0008091700042
:1004F0008093D10080917B008093D2008091F500A1
:100500008093D30080917C008093D40080916D0013
:100510008093D5008091B6008093D600F89401ECCA
:1005200010E0C1E0D1E0F80161918F01CE0199DCCA
:100530002196C731F1E0DF07B1F765EA80E091E08D
:1005400090DC7894DF91CF911F910F910895809165
:10055000D900853010F492E005C08E3010F491E09F
:1005600001C090E080E80FB6F89486BD96BD0FBE3E
:100570000895882321F0813029F4BC9804C0BC98E8
:10058000C4980895BC9AC49A0895CF93C82F8093B5
:10059000D9008093D8008091DA0081110AC091E0DF
:1005A000C11101C090E081E0C23408F480E0890FFD
:1005B000E0DFC11103C019BC18BC0DC0C1508C2FA5
:1005C00090E0FC01EF53FF4FE491E9BDFC01E55DD4
:1005D000FF4FE491E8BDCF91BACF8093BF00D5CF54
:1005E000CF93C091D90089E18C0F873908F080E062
:1005F000CCDF82E02BDE8C2FCF91C7CFCF93C09181
:10060000D90080E0C2DF83E021DE8C2FCF91BDCF07
:100610009091F8009D3110F480E006C08F70E82FB3
:10062000F0E0EC57FF4F8081A4CFCF93C0917900C9
:10063000C11149C0883039F41092BA001092B80044
:100640001092B70041C0813B59F48091BA008150AB
:100650008330C8F583E08093BA008093B90033C03B
:10066000853BA9F4CB016EE370E0CCDB892B61F50F
:100670008091BA008A3F40F58B5F8093BA008093E7
:10068000B9001092B8001092B700AADF1DC08130E7
:10069000D1F48091B7009091B800019688382EE08F
:1006A000920728F49093B8008093B7000DC0109281
:1006B000B8001092B7008091BA00882329F08150C9
:1006C0008093BA0001C0C1E08C2FCF910895FF92B2
:1006D0000F931F93CF93DF938C01EB01F42E809146
:1006E000F3009091F400892B31F0E091F300F09148
:1006F000F40089E009951093F4000093F300012BB6
:1007000039F0E091F300F091F400BE018F2D0995CE
:1007100081E08093C000DF91CF911F910F91FF90F6
:100720000895CF93DF93E091E200EE2359F0E1507A
:10073000E093E200F0E0EE0FFF1FED51FF4FC081AC
:10074000D18102C0C0E0D0E0E091E200EE2341F0B0
:10075000F0E0EE0FFF1FEF51FF4F8081918102C04B
:1007600080E090E04AE060E070E0B1DFCE01DF9130
:10077000CF910895883029F41092B3001092980018
:1007800015C08130F9F490919800911107C0603242
:10079000710528F1809398004FDD21C0913081F4DC
:1007A0006B3B710528F082E08093980080E016C0D2
:1007B00061157105A1F06270862F880F8E5E0EC0E4
:1007C000B0DF0DC0813859F481E0809398008091AA
:1007D000B3008F5F8093B3002FDD8BE4D6DE80E023
:1007E00008959C019091E200983088F4E92FF0E0A0
:1007F000EE0FFF1FED51FF4F318320839F5F9093DA
:10080000E20048E0C90163DF8091E20008958FEFC4
:1008100008950F931F93CF93DF93EC018B0181DF3A
:10082000B801CE01DF91CF911F910F91DACF8430C3
:1008300011F58091F3009091F4002AE08938920735
:1008400029F469E170E083E895E013C0835895408E
:1008500061F49091D900923040F0892F8695969559
:100860009695890FBADE80E0089560E070E08EE929
:1008700094E0CFDFF8CF81E00895813C29F460E077
:1008800070E08EE994E006C0823C31F460E070E0F4
:1008900084E694E0BEDF14C0813B41F4CB016EE3FB
:1008A00070E0B0DA892B61F49BDE0AC0813E51F41E
:1008B000CB016EE370E0A6DA6F5F60936C00D2DD6F
:1008C00080E0089581E00895CF93C0917900C1112F
:1008D00017C0813C29F460E070E08EE994E006C026
:1008E000823C31F460E070E084E894E092DF09C07B
:1008F000873B31F460E070E08BEA97E072DF01C083
:10090000C1E08C2FCF910895813C29F460E070E024
:100910008EE994E006C0823C31F460E070E08DE343
:1009200094E077DF07C0873B39F460E070E08FEA3E
:1009300097E057DF80E0089581E008950F931F93BB
:10094000CF938B01883079F480E01FDE80916D00B9
:1009500083700FDE1092BA00012B19F481E08093AE
:10096000DA00C0E0CBC0813051F469317105C8F3C1
:100970008093DA0080916D008370FBDDF2CF8330CD
:10098000F9F470939E0060939D0080916D008370D8
:10099000833011F4862F3CDEC0917900C111E1CF84
:1009A0008091B6008823E9F290E062EC71E00DDA04
:1009B00080179107B0F660E070E087EB97E08DC09C
:1009C000813B71F481E090E0B8DCDFDD8091BC0018
:1009D000811103C00831110520F261E070E037C0D9
:1009E000813ED9F38138B9F42091BE00222379F0F9
:1009F0008091BD0090E062EC71E0E7D940919D00EC
:100A000050919E004817590710F0822F02C0809124
:100A10007A0090E00EC0813C21F46091D90070E032
:100A200016C0823B61F4C0917900CC2329F086E99D
:100A300090E083DCAADD95CF86E9A7DD5FC0823E2A
:100A400011F480E0F7CF823C31F466E970E083E88E
:100A500095E0DFDE86CF8339A1F3833C29F460E0A3
:100A600070E084E694E0F5CF843C31F4B9DD60E0D9
:100A700070E087EB97E0EDCF8F3C29F460E070E009
:100A80008EE092E0E6CFC09179008A3B79F4672B43
:100A900069F4CC2329F0A4DD10927900E3DC61CF66
:100AA00060E070E083EA97E09CDE28C0C11125C0B9
:100AB0008A3C29F495DD81E0809379001CC0833B5A
:100AC00029F460E070E089E89AE007C0853C39F4D9
:100AD00087DD60E070E080E09CE09BDE0FC0873C3B
:100AE00061F490916D0081E0890F83709C7F982B59
:100AF00090936D003EDDB6DC01C0C1E08C2FCF913C
:100B00001F910F910895CF92DF92EF92FF920F9372
:100B10001F93CF93DF93182FEB01F0907800009193
:100B20007700D090BC00DD2019F0E090BB0002C03F
:100B3000EE24E394C090BA00BE01812F76DD60916F
:100B4000BA00662339F0C1100CC08091D90080939F
:100B50009C0007C0CC2029F060E070E08EE994E0B2
:100B60003AC0812F8D7F8830B9F41092B5001A30C9
:100B700019F4C0917A00D0E08F2D90E08C179D077A
:100B800030F410E0C017D10710F4C0937A00CE0102
:100B9000D4DB23DD81E070C0113CF1F2123C99F40A
:100BA00080917900811101C006E98091D9008017F8
:100BB00010F4802F02C080917A000FDD8091D9005F
:100BC00080939C0019C1143C41F480E0DEDC60E0BD
:100BD00070E087EB97E01DDE0FC18FE4810F82305C
:100BE00008F043C0DD2039F0CE0168E170E00AD999
:100BF000892B09F001C18091D900209761F4123B43
:100C000011F48FEF05C08017E0F7F816A8F081E027
:100C10008093650011C0C73391E0D90768F0801751
:100C200080F7CD36D24040F0F81630F0D9DC60E0E5
:100C300070E087EB97E0EDDDD091D9008091650001
:100C40006E2D70E0082E000C990BBFD88D0F911DF2
:100C500074DBC82F80937A00D81729F0813411F003
:100C6000081301C0CBDC8C2FA8CF8FE1810F82301D
:100C700030F480916500819580936500BDC011308E
:100C800009F08DC0EE9711F410936500662391F082
:100C900080919C0070E06150710990E096D860915D
:100CA000B90070E0C3D8611101C061E06093D80061
:100CB0006093BF002091D8003091D900822F90E03E
:100CC000831B910960919A0070919B006F5F7F4F29
:100CD00070939B0060939A00009709F48DC097FF72
:100CE00005C0383830F040E450E005C040E052E044
:100CF00002C040E051E05695479597FD01969595C5
:100D000087950097C1F74617570708F075C0231756
:100D100010F42FEF03C0321710F421E0230F7FEF00
:100D2000720F872F90E0AC014F535F4FFA0164912F
:100D3000731738F439B5311104C06F3F11F469BD30
:100D40000CC039B5361718F439B53F5F05C039B551
:100D5000631718F439B5315039BD855D9F4FFC01DB
:100D6000349168B5631718F438B53F5F05C068B5AE
:100D7000361718F438B5315038BD39B5FA014491F9
:100D8000341307C038B5FC018491381302C0209396
:100D9000D900DDDB10929B0010929A002DC0153017
:100DA000A1F48091D900823438F190E08C1B9D0B26
:100DB000282F813491052CF08739910518F026E908
:100DC00001C021E42093D80017C01630B9F49091E7
:100DD000D9008091BF00981778F4C90FD11D90E019
:100DE0008C179D0734F0C134D10524F4C1E4D0E060
:100DF00001C0EC01C093D80000E053C0173071F47B
:100E00009091D8008091D900891710F48F5F03C0AA
:100E1000981790F781508093D800EECF133C71F46F
:100E200081E0D11080E08093BC001CDBE7DB809187
:100E3000D90090E082DA80937A00BFCE00917900E9
:100E400001112EC0133B21F4CD2BB1F686E904C06D
:100E5000133E21F480917A00C0DB23C0153C41F49D
:100E600080E093DB60E070E080E09CE0D2DC19C0C1
:100E7000173B29F460E070E08DE997E00FC01A3C61
:100E800039F48091D9008093BE00ECDAA9DB09C067
:100E90001A3B31F460E070E087EA97E0A2DC01C021
:100EA00001E0802FDF91CF911F910F91FF90EF9084
:100EB000DF90CF900895883061F41092990080E01F
:100EC00064DB8091DB00811136C081E08093990062
:100ED00022C0982F907F903BB1F420919900421747
:100EE00078F0CB016DE570E08DD7029739F42F5F74
:100EF000209399004217F8F088E303C082E101C013
:100F000080E043DB18C0903E61F480919900882313
:100F100089F0481778F060E070E08AEB93E061DCDC
:100F20000AC08A3041F46091B30080919900F901C0
:100F3000099598DAF6DB80E008954091BC004E5F99
:100F40002AE531E0B8CF2AE531E043E0B4CF25E926
:100F500031E042E0B0CF20E132E041E0ACCF24E12B
:100F600032E042E0A8CF2FE232E041E0A4CF0F937D
:100F70001F93CF93DF93D82F8B0180798039B1F401
:100F800020917400909175008D2F8F70823041F404
:100F90008091BE00811108C0822F291728F403C058
:100FA000822F921708F4892FF0DA1BC0803819F4C9
:100FB00080E0EBDA08C0D83031F480916D0086957E
:100FC0008695D7DA39C0D13061F40931110508F4BA
:100FD00052C0D093DA0080916D0086958695C9DA6B
:100FE0004AC0D33049F480916D008C708C3009F088
:100FF00042C0802F0DDB3FC0D43C71F4C091BE00D5
:10100000CC2319F06C2F70E00EC060917A0070E074
:1010100083E895E0FEDB32C0D43B49F4E1DA10927C
:10102000370161E070E083E895E0F3DB24C0D53C54
:1010300019F466E970E0F7CFC0917900C1111DC0C5
:10104000DA3B31F460E070E083EB97E0CADB16C076
:10105000D73C99F490916D00892F869586958F5F86
:101060008370282F220F220F9370920F90936D00A0
:1010700080DAF8D903C0C0E001C0C1E08C2FDF9155
:10108000CF911F910F9108958CE287B910920201C0
:101090001092030186B1886486B908951092040104
:1010A00024B195B13091D7002295269526952370CD
:1010B000892F90E0880F991F880F991F820F911D2B
:1010C000830F8093D7008091F900882309F409C128
:1010D0001092F900809102019091DA00992319F0A1
:1010E000379810920201811141C080917D008823C0
:1010F00049F06091FE007091FF007093FB006093D7
:10110000FA0004C06091FA007091FB00605F7F4FAD
:10111000A6E076956795AA95E1F780E098E572D606
:1011200080917C00680F711D769567956093F8003B
:101130008091B200882311F0815007C06D3138F4DE
:1011400060E070E084E024D885E08093B200809174
:10115000DA008111BDC08FEA87B981E08093020176
:101160001092030186B1886486B9B2C0813009F05B
:10117000AFC080917D00811143C08091FC009091AF
:10118000FD0040969C0145E0369527954A95E1F78C
:10119000A091F500A901569547950A2E000CBB0BAE
:1011A000CD0183519140840F951F9093F700809358
:1011B000F6008091A100E82FF0E0EE0FFF1FEE5542
:1011C000FF4F40815181B901641B750B318320832E
:1011D0008F5F87708093A100CB01880F991F880FC4
:1011E000991F40917B0050E04D5E5E4F4A1B5B0BA8
:1011F000440F551F841B950B820F931F23E01CC0C7
:1012000080910001909101019093FD008093FC007A
:10121000409635E0969587953A95E1F7E2EAF0E059
:101220008193919320E0E23BF207D1F7A6CF00979C
:1012300009F00196215029F018161906C4F70197F4
:10124000F9CF18161906E4F477FD39C02091A000F3
:1012500012160CF1880F991FBC016350710977FFBA
:1012600002C06F5F7F4F759567951616170614F0CD
:1012700061E070E088E1861B8093A00085E026C0D5
:101280008C3F2FEF9207DCF477FF19C02091A0006C
:1012900027FF05C02450281B2093A00018C024EE6F
:1012A000281B2093A0002091F8002F3180F06CEFD4
:1012B0007FEF681B790B7595679586E007C0809175
:1012C000F8008E3120F060E070E087E061D7DCDE6E
:1012D00080917D00882329F080917D00815080934A
:1012E0007D0008950F931F93CF931092DD0080919E
:1012F0003501909136019C012F5F3F4F88279078F0
:10130000822B932B9093360180933501C091DB00A3
:10131000B3D7C81729F11092DA008093DB009091BF
:101320003701882359F0892F80699F709F3009F019
:101330008F5F8093370180E090E00DC0892F8F7E12
:1013400095FD02C0806801C0806C80933701809158
:101350003501909136016CD710923601109235010B
:1013600000913501109136018091DA00882379F0DF
:10137000B80183E00DD725D70F731127012B09F092
:1013800044C010929F0080DE87EE86B92EC0C091C7
:1013900037018C2F807F803B19F460E070E001C042
:1013A000B80181E0F5D6C4FF12C0C5FF02C0C80174
:1013B0000CC008311105C8F01092360110923501A9
:1013C000C062C093370180E090E032D70EC0CC23DA
:1013D00061F0C5FD09C00231110538F0C064C09349
:1013E000370180E090E024D727D780919F008111BA
:1013F00006C086B1886486B981E08093F900809147
:101400009F008F5F8F7180939F00CF911F910F91ED
:10141000089580910401811141DE8091DD008111E8
:1014200061CF0895CF92DF92EF92FF920F931F93B7
:10143000CF93DF93EC0110E800E088E0E82E87E02E
:10144000F82E92ECC92EDD24D394209709F18091D7
:10145000C00081111FC08091D900853040F482E026
:101460000FB6F89416BD86BD0FBEC60106C00FB6F6
:10147000F89416BD06BD0FBEC7010197F1F70FB670
:10148000F89416BD06BD0FBEC4DF9BD62197DDCFF5
:1014900081E001C080E0DF91CF911F910F91FF901B
:1014A000EF90DF90CF900895CF93C82F882381F0DD
:1014B00089E16BD886EA90E0B5DF80E066D88AEFF4
:1014C00090E0B0DFC150A1F78AE992E0CF91AACFB6
:1014D00089E15BD888E090E0A5DF80E056D88AEF0C
:1014E00090E0A0DFF1CFCF93DF9364E67FD4282F85
:1014F000892F6AE07BD4EC01222341F0822FD4DFD4
:101500008C2FD2DF8D2FDF91CF91CECFC111F8CFAD
:10151000F9CFDF92EF92FF920F931F93CF93DF9358
:10152000D82F8B01C0916B0081E08093B500C33050
:1015300009F0D3C0F090BA008D2F77D8FF2051F07A
:101540008091BA00811106C060E070E08EE994E0FD
:1015500060D9C3C0D83021F481E080936300BFC05C
:10156000D23C19F41092BA00C8C0D13BC1F490919A
:101570006200012B49F49E3610F08FEF03C09230C9
:1015800018F481E08093630080916300890F11F467
:1015900081E02BC18F3608F428C18EE626C1D13EEA
:1015A00031F480916300819580936300DCC0D23B6D
:1015B00061F481E08093630080916200823008F4DE
:1015C000DAC0815080936200D6C0D13009F0E4C007
:1015D0000E33110511F4D0936300D09097008D2D38
:1015E000880FD7FC809590E067E070E0EED3292F5C
:1015F000E09096008E2D880FE7FC8095D0916100D9
:101600006D2F70E090E0E1D3290FF09095008F2DC1
:10161000880FF7FC8095C09160006C2F70E090E01F
:10162000D4D3920F6091620070E0690F711D8091B8
:10163000BA00813091F48091B7009091B80025E014
:10164000969587952A95E1F724E730E0A901481B94
:10165000590BCA01BAD3B901D5D3862F96D700FD4D
:1016600005C013D68170D80ED09297008091940057
:10167000E80EE092960009D665E2B8D3F90EF09232
:10168000950003D68F7329F400D66DE0AFD3909305
:101690009400DD2331F0F9D58F7319F4D150D09334
:1016A0006100F3D5811107C0F0D56BE09FD3909313
:1016B000610010929600C33030F0E7D58F7119F4B5
:1016C000C150C0936000E1D58F7709F079C0DDD5B6
:1016D00066E08CD39093600073C0D83021F481E031
:1016E0008093640084C0D13C31F460E070E08EE906
:1016F00094E08FD87CC0D23C49F48C2F90E00196C6
:1017000065E070E093D380936B004BC0D13B49F50B
:10171000C23090F400FD6BC0EC2FF0E0E759FF4FB2
:10172000808190916400891B883020F08F3F91F573
:101730008EEF30C088E02EC0C43009F058C09091C0
:10174000680080916400890F823010F482E003C049
:10175000893708F088E7809368008091680015D782
:1017600046C0D13E31F4809164008195809364003D
:1017700018C0D23BA1F481E080936400C23060F5D0
:1017800000FD35C0EC2FF0E0E759FF4F80818F3F1F
:1017900071F18F5F80832BC0D13C09F4A6CFD23E7C
:1017A00011F460D624C0D53C39F460E070E080E0EC
:1017B0009CE02FD880E0D3CFD13011F081E018C069
:1017C0000E33110519F481E0809364008091D700F5
:1017D000080F0093D7000BC0C43049F48091680013
:1017E000833008F4BACF8150B6CF8093620080E096
:1017F000DF91CF911F910F91FF90EF90DF900895AF
:101800000F931F93CF93DF93D82F8B01883031F440
:101810008091B500813011F488E07BDE8D2F8079D6
:10182000803959F481E08093B400C091B500C111B2
:101830000AC080917A00A9D621C0803831F4109274
:10184000B40080E0A2D6C0E019C0D130B1F4C0919C
:10185000B400CC2351F08091B5008130A1F7B801DC
:10186000DF91CF911F910F9154CE0733114058F360
:10187000D093DA0080E07DD601C0C1E08C2FDF91EB
:10188000CF911F910F9108951F920F920FB60F9253
:1018900011242F933F938F939F93AF93BF93EF9315
:1018A000FF93809103018823E9F0E091020124B1C4
:1018B00035B1F0E0EE0FFF1FDF01A250BF4F2D93B7
:1018C0003C93E650FF4F808191818217930708F483
:1018D00001962817390708F401979183808381E0E6
:1018E0008093040181E080930301FF91EF91BF9108
:1018F000AF919F918F913F912F910F900FBE0F90BD
:101900001F9018951F920F920FB60F9211248F936C
:1019100081E08093DD008F910F900FBE0F901F909C
:1019200018951F920F920FB60F9211248F9381E09A
:101930008093DC008F910F900FBE0F901F90189531
:10194000F89484B7877F84BF0FB6F894A89581B5C3
:10195000886181BD11BC0FBEB89A81E083BF81EA66
:101960008ABDB99A88E088BB85BB8BB780628BBF84
:10197000A89581B5886181BD80E481BD85DB87EE56
:1019800086B9789481E062D460E070E087E194E009
:1019900028D71092C00024D66FD4811108C0F894C3
:1019A00080E091E056D2853A51F178948FC0C0E042
:1019B0008C2FEBD583E190E035DD8C2F8695E5D536
:1019C00083E190E02FDD58D4882381F0CF5FC034CD
:1019D00079F765E181E028D545D5C6E98C2FD5D5C5
:1019E00084E090E01FDDC150C9F7D9CFCC23B9F214
:1019F0008C2FCBD58DE090E015DDC150F7CF01ECF9
:101A000010E0C1E0D1E0CE0124D2F80181938F0132
:101A10002196C731F1E0DF07B1F778948091C100DA
:101A20008093BC008091C200809374008091C300B9
:101A3000809371008091C400809375008091C500EF
:101A4000809372008091C60080936F008091C700E0
:101A50008093BE008091C8008093BD008091C90032
:101A600080936B008091CA00809369008091CB00C5
:101A700080936A008091CC00809368008091CD00B3
:101A800080936C008091CE00809379008091CF008C
:101A9000809376008091D000809373008091D10074
:101AA000809370008091D20080937B008091D3005E
:101AB0008093F5008091D40080937C008091D500C4
:101AC00080936D008091D6008093B6008091BE0017
:101AD000811180937A0061E070E08EE994E081D614
:101AE00043E4342E52E0452E67EE562E70E4672E06
:101AF00077247394CC24C394D12CFCEF8F2EF3E085
:101B00009F2EAEE9AA2EA4E0BA2E5BD38091E0000E
:101B10009091E100009749F06091DE007091DF0044
:101B200078D61092E1001092E0008091DA008823CC
:101B300009F444C080E029D5A89581B5886181BDAC
:101B400031BC379899D38111FDCF76D38BB78062A2
:101B50008BBF109204011092DD001092DC00809186
:101B6000DA008823F9F085B7877E806185BF85B765
:101B7000806285BF889585B78F7D85BF8091DC00A9
:101B800081111092DA0080910401882329F070926B
:101B90007D007092F90082DA8091DD008823F9F2ED
:101BA000A1DBDDCF40927D008BB78F7D8BBF6CDAE0
:101BB00056B8A89581B5886181BD61BC2ADC1092B8
:101BC000C0008091F3009091F40022E08E309207E3
:101BD00079F4CEE1D0E0FE018491805365DC8CE2A3
:101BE00091E020DC2196F0E0CA32DF07A1F7B6C011
:101BF0002AE08938920779F03CE08030930709F0B9
:101C0000A2C08091B500813009F0D4C08091B400A9
:101C1000882309F4CFC0C0916B00C23001F120F0DD
:101C2000C43009F476C071CFEC2FF0E0E759FF4FD4
:101C3000D08186E9AAD4C11109C0DA3220F4C401E6
:101C40000197F1F707C081E090E003C08D2F8695E2
:101C500090E0E8DB80E099D48D2F90E0A9C015D307
:101C60008F73E82EF12C11D367E0C0D0E60102C0DB
:101C7000CC0FDD1F9A95E2F708D365E0B7D0F601E7
:101C800002C0EE0FFF1F9A95E2F7CE0FDF1FFDD2C5
:101C900090E0BE01CBD0C80FD91FC739D10514F0D1
:101CA000C6E9D0E08C2F71D4C701BCDB8E0133E0D4
:101CB000159507953A95E1F7011101C001E010E093
:101CC000C701B0DBC01BD10BD7FF02C0C0E0D0E022
:101CD0008C2F5BD4DAD2837031F4C701A3DBCE0141
:101CE0009595879552D4C230D10554F7CED26DE088
:101CF0007DD0E60102C0CC0FDD1F9A95E2F7C5D278
:101D000090E0BE017FD0C80FD91F80E03ED4CE0145
:101D10004FC0C0916800CC0FC73908F0C6E9D4E0C5
:101D20008C2F33D485E090E07DDB809168002DD44A
:101D300081E490E077DBD15099F780ED92E072DB9F
:101D400080E023D4E2CEF4E084369F0781F48091D2
:101D5000F800C9DB80917900882381F0B092E1001E
:101D6000A092E0001092DF001092DE00CECE24E0C0
:101D70008438920731F48091F600B5DB88EE93E069
:101D800017C08D539440B1F48091DB008111BDCE1A
:101D900080917A00FAD384E690E044DB80E0F5D3CA
:101DA00080916C0090E068EE73E00FD0845691094A
:101DB00039DBABCE85B7877E85BF85B7806285BFAF
:101DC000889585B78F7D85BFA0CE0024552704C098
:101DD000080E591F880F991F009729F0769567956F
:101DE000B8F37105B9F7802D952F0895991B79E007
:101DF00004C0991F961708F0961B881F7A95C9F79B
:101E000080950895AA1BBB1B51E107C0AA1FBB1FE9
:101E1000A617B70710F0A61BB70B881F991F5A9576
:101E2000A9F780959095BC01CD01089597FB072EE9
:101E300016F4009406D077FD08D0E4DF07FC05D047
:101E40003EF4909581959F4F0895709561957F4FD1
:101E50000895E199FECF9FBB8EBBE09A99278DB381
:101E60000895262FE199FECF9FBB8EBBE09A019784
:101E70000DB2021639F01CBA2DBB0FB6F894E29AD7
:0A1E8000E19A0FBE0895F894FFCF19
:101E8A00060B18010101000441294303020E000751
:101E9A0005787896010A0A780101412D0702740033
:101EAA0071006E0000010201000000000000010044
:041EBA000000000024
:00000001FF
